:020000040000FA
:020000002E28A8
:08000800A700030EA800241953
:10001000241C1528A4180F2885120516112805126E
:1000200085162208810024101A2823088100241430
:1000300005128512280E8300A70E270E0B1109004A
:10004000831285010730990083168501851183127B
:100050008316FF23900083128B1308002020831641
:100060008B018B1605308100811281118B17831251
:100070002411851405150030A200FE30A300851957
:100080003F280230A500FF30A600A608031DA503E7
:10009000A603A5080319A60803199B28851D452852
:1000A000A101C830A0008B13851D4528A00B542842
:1000B000851D5D28A10F58289B288B1721089B3E82
:1000C000031868282108643CA100A41424156C2896
:1000D0006430A102A41024152108FA3E03187128E7
:1000E00024112108A200643CA3002208FF3CA200C6
:1000F0002308FF3CA3002108FA3E03188D28291885
:10010000862829143230AA0005118D28AA0B8C28C4
:1001100005150130AA008D280511241D922885148B
:10012000A41C85102108F53E031C3F282910051545
:100130000130AA003F282411851405150130A500BF
:0A014000FF30A60085199B28452812
:02400E00943FDD
:00000001FF
